:10F800000C94387C0C94557C0C94557C0C94557C51
:10F810000C94557C0C94557C0C94557C0C94557C24
:10F820000C94557C0C94557C0C94557C0C94557C14
:10F830000C94557C0C94557C0C94557C0C94557C04
:10F840000C94557C0C94557C0C94557C0C94557CF4
:10F850000C94557C0C94557C0C94557C0C94557CE4
:10F860000C94557C0C94557C0C94557C0C94557CD4
:10F8700011241FBECFEFD0E1DEBFCDBF11E0A0E06D
:10F88000B1E0EAE5FFEF02C005900D92A030B107AC
:10F89000D9F712E0A0E0B1E001C01D92A930B10794
:10F8A000E1F70E944D7D0C94AC7F0C94007CCF93CB
:10F8B000DF93CDB7DEB724970FB6F894DEBF0FBE47
:10F8C000CDBF882309F481E020E0482F552741155A
:10F8D000510509F43DC0289A19821A821B821C82A4
:10F8E0000BC089819A81AB81BC810196A11DB11D9C
:10F8F00089839A83AB83BC8389819A81AB81BC81E4
:10F9000080589E43A040B04060F3289819821A8224
:10F910001B821C820BC089819A81AB81BC810196BC
:10F92000A11DB11D89839A83AB83BC8389819A8190
:10F93000AB81BC8180509A4FA040B04060F32F5FF4
:10F94000822F992787FD9095841795070CF4C3CFD4
:10F9500019821A821B821C8289819A81AB81BC81A7
:10F9600080509147A240B040A0F489819A81AB8138
:10F97000BC810196A11DB11D89839A83AB83BC8391
:10F9800089819A81AB81BC8180509147A240B0406F
:10F9900060F324960FB6F894DEBF0FBECDBFDF91A3
:10F9A000CF910895EF92FF920F931F93EE24FF24BF
:10F9B000870128988091C00087FD17C00894E11C3A
:10F9C000F11C011D111D81E0E81689E0F8068DE3A8
:10F9D000080780E0180770F3E0910001F091010141
:10F9E00009958091C00087FFE9CF289A8091C600D1
:10F9F000992787FD90951F910F91FF90EF900895A3
:10FA0000982F8091C00085FFFCCF9093C600089589
:10FA10000E94D27C803271F0809102018F5F8093CE
:10FA20000201853009F00895E0910001F091010193
:10FA30000995089584E10E94007D80E10E94007D87
:10FA40000895CF93C82F0E94D27C803241F08091DC
:10FA500002018F5F80930201853081F40AC084E146
:10FA60000E94007D8C2F0E94007D80E10E94007D1D
:10FA700005C0E0910001F09101010995CF91089531
:10FA8000282F90E007C08091C0008823E4F7809180
:10FA9000C6009F5F9217B8F30895CFEFD0E1DEBFA5
:10FAA000CDBF000094B714BE809160008861809340
:10FAB00060001092600091FF74C189E18093C400DE
:10FAC0001092C50088E18093C10086E08093C20057
:10FAD0005098589A209A83E00E94577C81E00E94B7
:10FAE000577C0E94D27C8033B9F18133C1F18034DC
:10FAF00009F456C0813409F45CC0823409F46EC044
:10FB0000853409F471C0803539F1813509F4F3C0C9
:10FB1000823511F1853509F4D3C0863509F4CBC09F
:10FB2000843609F465C0843709F4EBC0853709F4DD
:10FB3000D2C0863709F44AC0809102018F5F80935A
:10FB40000201853071F6E0910001F0910101099503
:10FB50000E94D27C803349F60E94087DC2CF0E9469
:10FB6000D27CC82F803241F784E10E94007D81E47D
:10FB70000E94007D86E50E94007D82E50E94007D56
:10FB80008C2F0E94007D89E40E94007D83E50E9405
:10FB9000007D80E50E94007D80E10E94007DA1CF74
:10FBA0000E94D27C8638C0F20E94D27C0E94087DDE
:10FBB00098CF0E94D27C803809F407C1813809F4BB
:10FBC00000C1823809F4F9C0883921F080E00E9430
:10FBD000217D87CF83E00E94217D83CF84E10E9435
:10FBE000407D0E94087D7DCF85E00E94407DF9CF59
:10FBF0000E94D27C809306020E94D27C80930502F0
:10FC0000809108028E7F809308020E94D27C853406
:10FC100009F44BC0E5E0F1E0119281E0E438F80727
:10FC2000D9F3D0F3C0E0D0E08091050290910602B4
:10FC30001816190678F405E011E00E94D27CF8014C
:10FC400081938F0121968091050290910602C81739
:10FC5000D90798F30E94D27C803209F06DCF809151
:10FC6000080280FFB6C0C0E0D0E0209105023091CC
:10FC7000060212161306B8F4E0910301F091040194
:10FC8000A5E0B1E0F999FECFF2BDE1BD8D9180BD57
:10FC9000FA9AF99A31962196C217D30798F3F093FE
:10FCA0000401E093030184E175CF80910802816033
:10FCB00080930802AFCF84E00E94407D80E087CF30
:10FCC0000E94D27C809303010E94D27C8093040125
:10FCD0000E94087D06CF0E94D27C803209F02CCF92
:10FCE00084E10E94007D8EE10E94007D86E90E94F1
:10FCF000007D89E04FCF0E94087D88E080936000FE
:10FD0000FFCF0E94D27C809306020E94D27C809317
:10FD100005020E94D27C853409F449C08091080212
:10FD20008E7F809308028091030190910401880FD7
:10FD3000991F90930401809303010E94D27C80322A
:10FD400009F0CFCE84E10E94007DC0E0D0E0209198
:10FD50000502309106021216130608F01DCFE0913D
:10FD60000301F09104018091080280FF96C0F99987
:10FD7000FECFF2BDE1BDF89A80B50E94007DE09112
:10FD80000301F09104013196F0930401E093030123
:10FD900020910502309106022196C217D30718F36D
:10FDA000FBCEE0910001F0910101099586CE809192
:10FDB0000802816080930802C0CF80E10E94217D0B
:10FDC00090CE81E00E94217D8CCE82E00E94217D38
:10FDD00088CE8091030190910401880F991F909320
:10FDE0000401809303018091050280FF09C0809186
:10FDF00005029091060201969093060280930502F7
:10FE0000F999FECF1127E0910301F0910401C5E0BB
:10FE1000D1E08091050290910602103091F400919A
:10FE2000570001700130D9F303E000935700E895C3
:10FE30000091570001700130D9F301E100935700A0
:10FE4000E895099019900091570001700130D9F39D
:10FE500001E000935700E8951395103898F01127AA
:10FE60000091570001700130D9F305E0009357006D
:10FE7000E8950091570001700130D9F301E100933A
:10FE80005700E8953296029709F0C7CF103011F06D
:10FE90000296E5CF112484E17DCE869580FF06C0D1
:10FEA0003196F0930401E093030176CF84910E9490
:10FEB000007D2091050230910602E0910301F0914E
:10FEC0000401EECF1F93CF930E94D27CC82F0E94D3
:10FED000007D0E94D27C182F0E94007DC1362CF03C
:10FEE000C75511363CF0175508C0C033D4F3C05382
:10FEF0001136CCF710330CF01053C295C07FC10FF0
:10FF00008C2F992787FD9095CF911F910895CF93BE
:10FF1000282F992787FD9095807F907095958795DC
:10FF20009595879595958795959587958A303CF019
:10FF3000895AC22FCF70CA303CF0C95A06C0805DC2
:10FF4000C22FCF70CA30CCF7C05D0E94007D8C2FCD
:0AFF50000E94007DCF910895FFCFBD
:040000030000F80001
:00000001FF
